:020000040000FA
:0400000023EF00F0FA
:020004000000FA
:040008000FEF00F006
:040018000FEF00F0F6
:04001C001000106E52
:10002000D838116EF2B402D01CEF00F04386282EAF
:1000300003D04484640E286E1138D86E103A1038FC
:10004000F294F28E10003FEC02F0416AF29EF29AB6
:10005000F294DDEC0CF0E9EC09F099EC04F067ECBB
:1000600004F069EC02F09488948C93808A988B8ACF
:10007000BEEC09F0BEEC09F082A809D08B9ABEEC68
:1000800009F0BEEC09F082B802D0439001D0438061
:100090008B9A8B8EBEEC09F0BEEC09F082AC09D0D5
:1000A0008B9EBEEC09F0BEEC09F082BC02D04392FC
:1000B00001D043828B9E8A82BEEC09F0BEEC09F02F
:1000C00081A009D08A92BEEC09F0BEEC09F081B0A3
:1000D00002D0439401D043848A92939E938C8A8E5B
:1000E00062EC02F081AC25D08A9E62EC02F081BC09
:1000F00020D08A8E62EC02F081AC1BD08A9E62EC2A
:1001000002F081BC16D08A8E62EC02F081AC11D074
:100110008A9E62EC02F081BC0CD000D0000EA96E69
:1001200083EC04F0A850E87EA86E000EA96E8AEC5D
:1001300004F03FEC02F088EC0CF0D9EC09F067EC2D
:100140000DF0C6EC0BF0D9EC09F067EC0DF006EC05
:100150000CF0D9EC09F067EC0DF02EEC0CF0F0ECA3
:1001600002F067EC0DF0000EA96E83EC04F0A850CD
:10017000E8AECAD04FEC0BF0D9EC09F067EC0DF00B
:10018000939E938C456A8BEC03F08A8E62EC02F0AE
:1001900081AC34D08A9E62EC02F081BC2FD08A8E72
:1001A00062EC02F081AC2AD08A9E62EC02F081BC43
:1001B00025D08A8E62EC02F081AC20D08A9E62EC5F
:1001C00002F081BC1BD0640E3B26000E3C220F0EB9
:1001D0003C6401D006D03C6207D0A00E3B6404D042
:1001E00000D03C6A640E3B6ED9EC03F0456AC9EC62
:1001F00009F0C9EC09F0C9EC09F0C7D7452A230E6C
:100200004562C3D767EC04F0040EA96E83EC04F0DA
:10021000A8503B6208D0050EA96E83EC04F0A850EC
:100220003C6201D00ED03BC0A8FF040EA96E8AEC40
:1002300004F03CC0A8FF050EA96E8AEC04F099EC0E
:1002400004F067EC0DF0939E938C456A18EC03F074
:100250008A8E62EC02F081AC34D08A9E62EC02F0AD
:1002600081BC2FD08A8E62EC02F081AC2AD08A9EAB
:1002700062EC02F081BC25D08A8E62EC02F081AC87
:1002800020D08A9E62EC02F081BC1BD00A0E1E2692
:10029000000E1F22010E1F6401D006D01F6207D07E
:1002A000F40E1E6404D000D01F6A0A0E1E6E69ECA4
:1002B00003F0456AC9EC09F0C9EC09F0C9EC09F092
:1002C000C7D7452A230E4562C3D769EC02F0010E59
:1002D000A96E83EC04F0A8501E6208D0020EA96E2D
:1002E00083EC04F0A8501F6201D00ED01EC0A8FFFE
:1002F000010EA96E8AEC04F01FC0A8FF020EA96EC1
:100300008AEC04F099EC04F067EC04F069EC02F07C
:10031000938E938C9CEC0AF043A401D003D0080E7A
:10032000326E03D0040E326E00D043A201D003D04F
:10033000040E316E03D0020E316E00D0F28E010E2B
:10034000C26E75EC06F048C021F047C020F0050EE3
:10035000C26E75EC06F048C023F047C022F043B0EF
:1003600036D021C017F020C016F023C015F022C0EF
:1003700014F02450165E2550175AD8B003D0176ACF
:10038000166A0ED00F0E176401D006D0176206D081
:10039000A00E166403D000D0438C02D0439C00D042
:1003A0002650145E2750155AD8B003D0156A146A27
:1003B00044D00F0E156401D006D0156206D0A00EF1
:1003C000146403D000D0438A38D0439A36D021C079
:1003D00015F020C014F023C017F022C016F02450EE
:1003E000145E2550155AD8B003D0156A146A0ED081
:1003F0000F0E156401D006D0156206D0A00E14644D
:1004000003D000D0438A02D0439A00D02650165E13
:100410002750175AD8B003D0176A166A0ED00F0E9D
:10042000176401D006D0176206D0A00E166403D060
:1004300000D0438C02D0439C00D043B60CD044B4CF
:10044000F0EC02F0E0EC07F08EEC02F080AC76D736
:10045000FCEC03F073D7439695EC05F0FDEC05F04A
:1004600080AC01D007D0B2EC04F09EEC08F016ECA2
:1004700005F064D7FCEC03F061D73DEF02F07C0E91
:10048000D36E9B8C000E936E020E946E4F0E926E86
:100490008A6A8B6A898E0C0EBD6E040ECA6EFF0EC0
:1004A000CB6E000EBE6EBD9ABD98010EC26E3B0EA5
:1004B000C16E8D0EC06E950ED56EF26AF28EF28A06
:1004C000F28C1200BEEC09F0BEEC09F0BEEC09F0B3
:1004D0001200020EA96E83EC04F0A8CF57F0010EB3
:1004E000A96E83EC04F0A8CF56F0270E596E100EBB
:1004F000586E9CEC07F05DC051F05CC050F05BC0E2
:100500004FF05AC04EF0030E4B6EFF0E4A6EBDEC1C
:1005100007F04FC01DF04EC01CF0120019C057F07C
:1005200018C056F0270E596E100E586E9CEC07F04E
:100530005DC051F05CC050F05BC04FF05AC04EF04F
:100540001DC04BF01CC04AF0BDEC07F0080E336232
:1005500007D0030E4B6EE80E4A6EBDEC07F014D0C8
:10056000040E336207D0000E4B6E640E4A6EBDEC73
:1005700007F00AD0020E336207D0000E4B6E0A0E4F
:100580004A6EBDEC07F000D0030E4F6401D006D0D8
:100590004F6209D0FF0E4E6406D000D0030E4F6E9E
:1005A000FF0E4E6E00D04EA004D00F01BD8800019A
:1005B00004D000000F01BD9800014EA204D00F012D
:1005C000BD8A000104D000000F01BD9A0001D8903F
:1005D0004F324E32D8904F324E324EC0BEFF1200D4
:1005E0008B86C9EC09F0C9EC09F0C9EC09F0C9EC3B
:1005F00009F0C9EC09F0010EC26E75EC06F048C0B6
:1006000025F047C024F0050EC26E75EC06F048C018
:1006100027F047C026F08B96C9EC09F0C9EC09F029
:10062000C9EC09F0C9EC09F0C9EC09F044941200D6
:10063000010E2FEC0DF0410E06EC0DF06E0E06ECE7
:100640000DF0610E06EC0DF06C0E06EC0DF0050ED3
:1006500006EC0DF0670E06EC0DF0200E06EC0DF02A
:100660006B0E06EC0DF0690E06EC0DF06D0E06EC4F
:100670000DF0650E06EC0DF06E0E06EC0DF0650E3D
:1006800006EC0DF0740E06EC0DF0400E2FEC0DF0A4
:10069000760E06EC0DF0010E06EC0DF0670E06EC82
:1006A0000DF06B0E06EC0DF0690E06EC0DF0740EFD
:1006B00006EC0DF0010E06EC0DF0720E06EC0DF0DE
:1006C000010E06EC0DF0730E06EC0DF03A0E06EC82
:1006D0000DF04C0E2FEC0DF01FC012F01EC013F0E9
:1006E00061EC07F02A6601D005D0300E2A2406EC12
:1006F0000DF005D0200E2A2406EC0DF000D0300EAF
:100700002B2406EC0DF0300E2C2406EC0DF0570EC9
:1007100006EC0DF01200010E2FEC0DF0560E06EC5B
:100720000DF06F0E06EC0DF06E0E06EC0DF0610E86
:1007300006EC0DF06C0E06EC0DF06B0E06EC0DF0F9
:10074000690E06EC0DF06A0E06EC0DF0650E06EC77
:100750000DF06C0E06EC0DF07A0E06EC0DF0010EAD
:1007600006EC0DF0730E06EC0DF0400E2FEC0DF0C4
:10077000760E06EC0DF0010E06EC0DF0670E06ECA1
:100780000DF06B0E06EC0DF0690E06EC0DF0740E1C
:1007900006EC0DF0010E06EC0DF0720E06EC0DF0FD
:1007A000010E06EC0DF0730E06EC0DF03A0E06ECA1
:1007B0000DF04B0E2FEC0DF03CC012F03BC013F0CF
:1007C00061EC07F0296601D005D0300E292406EC33
:1007D0000DF005D0200E292406EC0DF000D0300ECF
:1007E0002A2406EC0DF0300E2B2406EC0DF0300E12
:1007F0002C2406EC0DF0120043AC01D030D0040ED6
:10080000326206D016503B5C17503C5828E332D079
:10081000080E326212D00A0E4A6E000E4B6E16C0DF
:100820004EF017C04FF0506A516ABDEC07F04E50C1
:100830003B5C4F503C5813E31DD0640E4A6E000ED3
:100840004B6E16C04EF017C04FF0506A516ABDECA7
:1008500007F04E503B5C4F503C5801E30BD0400E2C
:100860002FEC0DF0140E386E050E06EC0DF0382E40
:10087000FBD7120017C036F016C035F0400E2FEC33
:100880000DF0376A100E386E3950355CD8B001D093
:1008900007D0356E050E06EC0DF0382EF5D7120098
:1008A0003606D8B0F6D700D0366A3A50355ED8B0A2
:1008B00001D002D0372AF8D7375006EC0DF0382E89
:1008C00001D01200000E06EC0DF0F9D71200100E48
:1008D0004A6E000E4B6E3BC04EF03CC04FF0506A6B
:1008E000516ABDEC07F04EC039F0050E4A6E000E9D
:1008F0004B6E39C04EF04F6A506A516ABDEC07F03A
:100900004EC03AF01200A69EA69CA680A6B086EF26
:1009100004F01200A69EA69CA684F29E550EA76E19
:10092000AA0EA76EA682F28EA6B294EF04F0A69449
:100930001200010EA96E83EC04F0A8CF1EF0020E87
:10094000A96E83EC04F0A8CF1FF0040EA96E83EC0F
:1009500004F0A8CF3BF0050EA96E83EC04F0A8CFFD
:100960003CF0120019C012F018C013F061EC07F04F
:10097000000E336204D0410E2FEC0DF004D0400E77
:100980002FEC0DF000D0296606D033B604D0200E2F
:1009900006EC0DF004D0300E292406EC0DF033A641
:1009A00004D02E0E06EC0DF000D02A660AD033B625
:1009B00008D033B406D0296604D0200E06EC0DF022
:1009C00004D0300E2A2406EC0DF033A404D02E0EF1
:1009D00006EC0DF000D02B660ED033B60CD033B43D
:1009E0000AD033B208D0296606D02A6604D0200E79
:1009F00006EC0DF004D0300E2B2406EC0DF033A2E3
:100A000004D02E0E06EC0DF000D0300E2C2406EC97
:100A10000DF0570E06EC0DF0200E06EC0DF0200E3A
:100A200006EC0DF0200E06EC0DF0120044B003D0E1
:100A300043B801D019D0490E2FEC0DF0200E06EC72
:100A40000DF0200E06EC0DF0200E06EC0DF03E0E23
:100A500006EC0DF0310E06EC0DF06B0E06EC0DF011
:100A6000060E06EC0DF01200000E346204D04A0EA1
:100A70002FEC0DF004D0490E2FEC0DF000D02D66B8
:100A800006D034B604D0200E06EC0DF004D0300EA3
:100A90002D2406EC0DF034A604D02E0E06EC0DF03D
:100AA00000D02E660AD034B608D034B406D02D66F5
:100AB00004D0200E06EC0DF004D0300E2E2406ECEF
:100AC0000DF034A404D02E0E06EC0DF000D02F66ED
:100AD0000ED034B60CD034B40AD034B208D02D665F
:100AE00006D02E6604D0200E06EC0DF004D0300E99
:100AF0002F2406EC0DF034A204D02E0E06EC0DF0DF
:100B000000D0300E302406EC0DF043A807D06B0E59
:100B100006EC0DF0060E06EC0DF01200060E06ECCB
:100B20000DF0200E06EC0DF0120015C012F014C0EE
:100B300013F061EC07F0000E2FEC0DF043AA13D078
:100B4000200E06EC0DF02D0E06EC0DF02D0E06EC31
:100B50000DF02D0E06EC0DF02D0E06EC0DF0560EE0
:100B600006EC0DF01200296606D031B604D0200E36
:100B700006EC0DF004D0300E292406EC0DF031A661
:100B800004D02E0E06EC0DF000D02A660AD031B645
:100B900008D031B406D0296604D0200E06EC0DF042
:100BA00004D0300E2A2406EC0DF031A404D02E0E11
:100BB00006EC0DF000D02B660ED031B60CD031B45F
:100BC0000AD031B208D0296606D02A6604D0200E99
:100BD00006EC0DF004D0300E2B2406EC0DF031A203
:100BE00004D02E0E06EC0DF000D0300E2C2406ECB6
:100BF0000DF0560E06EC0DF0120017C012F016C0E4
:100C000013F061EC07F0090E2FEC0DF043AC16D099
:100C1000200E06EC0DF02D0E06EC0DF02D0E06EC60
:100C20000DF02D0E06EC0DF02D0E06EC0DF0410E24
:100C300006EC0DF0200E06EC0DF01200296606D031
:100C400032B604D0200E06EC0DF004D0300E29246C
:100C500006EC0DF032A604D02E0E06EC0DF000D0FE
:100C60002A660AD032B608D032B406D0296604D03B
:100C7000200E06EC0DF004D0300E2A2406EC0DF008
:100C800032A404D02E0E06EC0DF000D02A660ED051
:100C900032B60CD032B40AD032B208D0296606D0AF
:100CA0002A6604D0200E06EC0DF004D0300E2B2462
:100CB00006EC0DF032A204D02E0E06EC0DF000D0A2
:100CC000300E2C2406EC0DF0020E326207D06D0EB1
:100CD00006EC0DF0410E06EC0DF01200410E06EC94
:100CE0000DF0200E06EC0DF01200500E456E01EED8
:100CF00000F0C280A8EC09F0C282C2B27DEF06F01B
:100D0000C3CFEEFFC4CFEEFF452EF6D7466A01EE05
:100D100001F011EE03F0EF50E76401D01BD0E76261
:100D200009D0ED52E552EF50E76401D018D0E652F9
:100D3000EE5200D0E652E652010EE2622CD0A10E35
:100D4000E162E9D700D0ED6AEE6A462A080E4662F3
:100D5000DED70CD0E1CFE9FFE2CFEAFFEBD7E1CF5E
:100D6000E9FFE2CFEAFFEE52E652E4D7466A01EE2F
:100D700001F011EE03F0EF660ED0ED52EE660BD0EF
:100D8000EE52EE52E652E652010EEA62F4D79F0EA0
:100D9000E962F1D70ED0E76613D0E552E66610D0CF
:100DA000E652E652010EE262F6D7A10EE162F3D7F7
:100DB00000D0ED6AEE6A462A080E4662D8D71BD0EC
:100DC000EF50E76001D00BD0E762EAD7ED52E55271
:100DD000EF50E76001D008D0E652EE52E1D7E1CF04
:100DE000E9FFE2CFEAFFDCD7E1CFE9FFE2CFEAFF9C
:100DF000EE52E652D5D7476A486A496A500E466EA7
:100E000001EE00F0EE504726EE504822D8A001D067
:100E1000492A46064666F6D7200E4726000E482287
:100E2000000E4922D890493248324732D890493290
:100E300048324732D890493248324732D890493206
:100E400048324732D890493248324732D8904932F6
:100E500048324732120030D8F36ED8900BD020EED3
:100E600000F0330EDF26DFB6F00BDFBE0F0BDE5EC9
:100E7000D9A4F7D7053606360736003601360236CE
:100E80000336F32EECD703380F0B0F6E03500F0B06
:100E90000E6E02380F0B0D6E02500F0B0C6E0138E8
:100EA0000F0B0B6E01500F0B0A6E00380F0B096E03
:100EB00000500F0B086E1200006A016A026A036A92
:100EC000180C296A2A6A2B6A2C6A030E125CE80E37
:100ED000D8B4135CD8A07FEF07F0030E125CD8A043
:100EE0007FEF07F076EF07F07FEF07F0126EE80E66
:100EF000135C136ED8A01206292A65EF07F0640E62
:100F0000135CD8B08AEF07F0126688EF07F08EEF17
:100F100007F01206136E2A2A7FEF07F00A0E135C01
:100F2000D8A099EF07F02B2A136E8EEF07F013C0AD
:100F30002CF013C02CF012005A6A5B6A5C6A5D6A7E
:100F400058505602F3CF5AF0F4CF5BF05950570285
:100F5000F3CF5CF0F4CF5DF058505702F3505B26AE
:100F6000F4505C22E86A5D2259505602F3505B2629
:100F7000F4505C22E86A5D221200200E526E4D6A27
:100F80004C6AD8904E364F36503651364C364D3628
:100F9000D8B0D5EF07F04B504D5CD8A4D2EF07F096
:100FA0004A504C5CD8A0DCEF07F04A504C5ED8A009
:100FB0004D064B504D5E4E80522EC1EF07F0120091
:100FC00015C057F014C056F017C059F016C058F0AD
:100FD0009CEC07F07F0E526E960E536E980E546E78
:100FE000000E556E5A50525C5B5053585C5054582A
:100FF0005D50555801E207D0080E316251D0020E03
:1010000032624ED000D0880E5A26130E5B22000E9C
:101010005C22000E5D22100E4A6E270E4B6E5AC0E7
:101020004EF05BC04FF05CC050F05DC051F0BDECC5
:1010300007F04FC019F04EC018F0080E31620FD003
:10104000020E326203D0080E336E77D0080E326281
:1010500003D0040E336E71D0020E336E6ED0040EC8
:1010600031620FD0020E326203D0040E336E65D0AF
:10107000080E326203D0020E336E5FD0020E336E62
:101080005CD0020E326203D0020E336E56D0080ED0
:10109000326203D0020E336E50D0000E336E4DD04C
:1010A000F40E5A26010E5B22000E5C22000E5D2219
:1010B000E80E4A6E030E4B6E5AC04EF05BC04FF006
:1010C0005CC050F05DC051F0BDEC07F04FC019F0AE
:1010D0004EC018F0080E31620FD0020E326203D0FB
:1010E000080E336E2AD0080E326203D0080E336E1B
:1010F00024D0040E336E21D0040E31620FD0020EC4
:10110000326203D0080E336E18D0080E326203D05C
:10111000040E336E12D0020E336E0FD0020E326206
:1011200003D0040E336E09D0080E326203D0020ED3
:10113000336E03D0000E336E00D01200176604D059
:10114000166602D04480120044904398100E346E0C
:10115000080E316204D03446344634460BD0040EB7
:10116000316203D03446344605D0020E316202D0DB
:10117000344600D0080E326204D034423442344245
:101180000ED0040E326203D03442344208D0020E34
:101190003262FDD7344234423442344200D015C06A
:1011A00057F014C056F0270E596E100E586E9CEC76
:1011B00007F0800E346201D00CD0400E346201D0B2
:1011C00023D0200E346201D039D0100E346267D0A3
:1011D0004ED0270E4B6E100E4A6E5AC04EF05BC0BA
:1011E0004FF05CC050F05DC051F0BDEC07F04EC058
:1011F0005AF04FC05BF050C05CF051C05DF034421B
:101200003442344234424BD0030E4B6EE80E4A6EE9
:101210005AC04EF05BC04FF05CC050F05DC051F062
:10122000BDEC07F04EC05AF04FC05BF050C05CF010
:1012300051C05DF034423442344231D0000E4B6E26
:10124000640E4A6E5AC04EF05BC04FF05CC050F066
:101250005DC051F0BDEC07F04EC05AF04FC05BF0DE
:1012600050C05CF051C05DF03442344218D0000EE2
:101270004B6E0A0E4A6E5AC04EF05BC04FF05CC017
:1012800050F05DC051F0BDEC07F04EC05AF04FC0B9
:101290005BF050C05CF051C05DF0344200D017C02C
:1012A0004BF016C04AF05AC04EF05BC04FF05CC025
:1012B00050F05DC051F0BDEC07F050C007F04FC0DA
:1012C00006F04EC005F02BEC07F00F6601D00BD0F6
:1012D0000FC02DF00EC02EF00DC02FF00CC030F05E
:1012E0003442438834D00E6601D00AD00EC02DF0AF
:1012F0000DC02EF00CC02FF00BC030F0438827D06B
:101300000D6601D00CD00DC02DF00CC02EF00BC01E
:101310002FF00AC030F034423442439818D00C66A3
:1013200001D00BD00CC02DF00BC02EF00AC02FF056
:1013300009C030F0344243980AD00BC02DF00AC0E7
:101340002EF009C02FF008C030F0439800D01200F2
:10135000020E3F6E290E3E6E3E2EACEF09F03F2E80
:10136000ACEF09F012000C0E3F6EAE0E3E6E3E2E3C
:10137000B7EF09F03F2EB7EF09F01200750E3F6E80
:10138000E00E3E6E3E2EC2EF09F03F2EC2EF09F096
:101390001200050E406E910E3F6ECF0E3E6E3E2E39
:1013A000CFEF09F03F2ECFEF09F0402ECFEF09F03D
:1013B00012002E0E406EA90E3F6E2E0E3E6E3E2E79
:1013C000DFEF09F03F2EDFEF09F0402EDFEF09F0ED
:1013D000120067EC0DF0400E4CEC0DF0000E06EC28
:1013E0000DF00A0E06EC0DF0000E06EC0DF00E0EE0
:1013F00006EC0DF0110E06EC0DF0110E06EC0DF0E2
:101400000E0E06EC0DF0000E06EC0DF0020E06ECD2
:101410000DF0040E06EC0DF00E0E06EC0DF0110EA4
:1014200006EC0DF01F0E06EC0DF0100E06EC0DF0A4
:101430000E0E06EC0DF0000E06EC0DF0020E06ECA2
:101440000DF0040E06EC0DF0000E06EC0DF00C0E87
:1014500006EC0DF0040E06EC0DF0040E06EC0DF09B
:101460000E0E06EC0DF0000E06EC0DF0050E06EC6F
:101470000DF00A0E06EC0DF0000E06EC0DF00E0E4F
:1014800006EC0DF0110E06EC0DF0110E06EC0DF051
:101490000E0E06EC0DF0000E06EC0DF00A0E06EC3A
:1014A0000DF0000E06EC0DF0110E06EC0DF0110E15
:1014B00006EC0DF0110E06EC0DF0110E06EC0DF021
:1014C0000E0E06EC0DF0000E06EC0DF0020E06EC12
:1014D0000DF0040E06EC0DF0000E06EC0DF00E0EF5
:1014E00006EC0DF0110E06EC0DF0110E06EC0DF0F1
:1014F0000E0E06EC0DF0000E06EC0DF0020E06ECE2
:101500000DF0040E06EC0DF00E0E06EC0DF0110EB3
:1015100006EC0DF01F0E06EC0DF0110E06EC0DF0B2
:10152000110E06EC0DF0000E06EC0DF0000E2FEC87
:101530000DF067EC0DF0120067EC0DF0400E4CEC76
:101540000DF0000E06EC0DF0000E06EC0DF0000E96
:1015500006EC0DF0000E06EC0DF0000E06EC0DF0A2
:10156000000E06EC0DF0000E06EC0DF0000E06EC81
:101570000DF0100E06EC0DF0100E06EC0DF0100E36
:1015800006EC0DF0100E06EC0DF0100E06EC0DF052
:10159000100E06EC0DF0100E06EC0DF0100E06EC21
:1015A0000DF0180E06EC0DF0180E06EC0DF0180EEE
:1015B00006EC0DF0180E06EC0DF0180E06EC0DF012
:1015C000180E06EC0DF0180E06EC0DF0180E06ECD9
:1015D0000DF01C0E06EC0DF01C0E06EC0DF01C0EB2
:1015E00006EC0DF01C0E06EC0DF01C0E06EC0DF0DA
:1015F0001C0E06EC0DF01C0E06EC0DF01C0E06EC9D
:101600000DF01E0E06EC0DF01E0E06EC0DF01E0E7B
:1016100006EC0DF01E0E06EC0DF01E0E06EC0DF0A5
:101620001E0E06EC0DF01E0E06EC0DF01E0E06EC66
:101630000DF01F0E06EC0DF01F0E06EC0DF01F0E48
:1016400006EC0DF01F0E06EC0DF01F0E06EC0DF073
:101650001F0E06EC0DF01F0E06EC0DF01F0E06EC33
:101660000DF0000E06EC0DF0000E06EC0DF00E0E67
:1016700006EC0DF0110E06EC0DF0110E06EC0DF05F
:101680000A0E06EC0DF01B0E06EC0DF0000E06EC3B
:101690000DF0000E2FEC0DF067EC0DF0120025C0E0
:1016A00012F024C013F061EC07F0000E2FEC0DF0E7
:1016B000410E06EC0DF04E0E06EC0DF0300E06EC71
:1016C0000DF0200E06EC0DF06F0E06EC0DF0660E20
:1016D00006EC0DF0660E06EC0DF0730E06EC0DF048
:1016E000650E06EC0DF0740E06EC0DF03A0E06ECED
:1016F0000DF0200E06EC0DF02B50300F06EC0DF027
:101700002C50300F06EC0DF06D0E06EC0DF0560E61
:1017100006EC0DF027C012F026C013F061EC07F0C4
:10172000400E2FEC0DF0410E06EC0DF04E0E06ECC7
:101730000DF0310E06EC0DF0200E06EC0DF06F0EE4
:1017400006EC0DF0660E06EC0DF0660E06EC0DF0E4
:10175000730E06EC0DF0650E06EC0DF0740E06EC43
:101760000DF03A0E06EC0DF0200E06EC0DF02B50AD
:10177000300F06EC0DF02C50300F06EC0DF06D0E16
:1017800006EC0DF0560E06EC0DF01200000E2FECDC
:101790000DF0500E06EC0DF0490E06EC0DF0430E68
:1017A00006EC0DF02D0E06EC0DF0650E06EC0DF0BE
:1017B000730E06EC0DF0200E06EC0DF0700E06EC2C
:1017C0000DF0610E06EC0DF06E0E06EC0DF0650EE0
:1017D00006EC0DF06C0E06EC0DF06D0E06EC0DF047
:1017E000010E06EC0DF0720E06EC0DF0030E06EC89
:1017F0000DF0470E2FEC0DF0490E06EC0DF0490EE2
:1018000006EC0DF02E0E06EC0DF01200420E2FEC41
:101810000DF0760E06EC0DF0650E06EC0DF0720E76
:1018200006EC0DF07A0E06EC0DF0690E06EC0DF0EC
:10183000050E06EC0DF03A0E06EC0DF0020E300F20
:1018400006EC0DF02E0E06EC0DF0010E300F06EC3E
:101850000DF0000E300F06EC0DF01200010E2FEC13
:101860000DF0700E06EC0DF0610E06EC0DF02D0E75
:1018700006EC0DF0650E06EC0DF06C0E06EC0DF0AE
:10188000650E06EC0DF06B0E06EC0DF0740E06EC1A
:101890000DF0720E06EC0DF06F0E06EC0DF06E0EF4
:1018A00006EC0DF0690E06EC0DF06B0E06EC0DF07B
:1018B000610E06EC0DF0430E2FEC0DF0020E300F12
:1018C00006EC0DF0000E300F06EC0DF0010E300F9F
:1018D00006EC0DF0010E300F06EC0DF02E0E06ECAE
:1018E0000DF0000E300F06EC0DF0050E300F06EC7B
:1018F0000DF02E0E06EC0DF0010E300F06EC0DF083
:10190000050E300F06EC0DF02E0E06EC0DF0120059
:10191000410E06EC0DF0640E06EC0DF06A0E06ECBE
:101920000DF06F0E06EC0DF06E0E06EC0DF0200EB5
:1019300006EC0DF0610E06EC0DF07A0E06EC0DF0E3
:10194000200E06EC0DF0490E06EC0DF0730E06ECC1
:101950000DF0740E06EC0DF0650E06EC0DF06E0E3B
:1019600006EC0DF02C0E06EC0DF0420E2FEC0DF0F7
:10197000730E06EC0DF07A0E06EC0DF0650E06EC1B
:101980000DF0620E06EC0DF0620E06EC0DF0200E6E
:1019900006EC0DF06A0E06EC0DF0000E06EC0DF0F4
:1019A000760E06EC0DF0030E06EC0DF0740E06EC50
:1019B0000DF0210E06EC0DF01200C9EC09F0C9EC97
:1019C00009F0C9EC09F0C9EC09F0C9EC09F08A9AF0
:1019D0008A988B988B9A8B9C8B9E8A808A828A9419
:1019E0008A96BEEC09F08A88BEEC09F08A988B983A
:1019F0008B9A8B8C8B8E8A808A828A948A96BEEC94
:101A000009F08A88BEEC09F08A981200F2AE01D083
:101A100002D0449201D04482F29E8A988A8A8A96A1
:101A20008A948A928A908B9E8B9C8B9A8B98E8B032
:101A30008A86E8B28A84E8B48A82E8B68A80E8B8FE
:101A40008B8EE8BA8B8CE8BC8B8AE8BE8B888A8840
:101A5000A8EC09F08A9844A21200F28E12008A982B
:101A60008A9A8A968A948A928A908B9E8B9C8B9A69
:101A70008B88E8B08A86E8B28A84E8B48A82E8B6BD
:101A80008A80E8B88B8EE8BA8B8CE8BC8B8A8A880F
:101A9000A8EC09F08A9812008A988A9A8A968A9401
:101AA0008A928A908B9E8B9C8B8A8B98E8B08A86D0
:101AB000E8B28A84E8B48A82E8B68A80E8B88B8E75
:101AC000E8BA8B8C8A88A8EC09F08A9812008A9868
:101AD0008A9A8A868A948A928A908B9E8B9C8B9A09
:101AE0008B988A88A8EC09F08A98B3EC09F0B3ECDB
:101AF00009F01200000E2FEC0DF0200E06EC0DF098
:101B000006EC0DF006EC0DF006EC0DF006EC0DF019
:101B100006EC0DF006EC0DF006EC0DF006EC0DF009
:101B200006EC0DF006EC0DF006EC0DF006EC0DF0F9
:101B300006EC0DF006EC0DF006EC0DF01200400E78
:101B40002FEC0DF0200E06EC0DF006EC0DF006EC7F
:101B50000DF006EC0DF006EC0DF006EC0DF006ECC9
:101B60000DF006EC0DF006EC0DF006EC0DF006ECB9
:101B70000DF006EC0DF006EC0DF006EC0DF006ECA9
:0C1B80000DF006EC0DF01200C4EF0DF0AB
:020000040030CA
:0100010038C6
:01000200F904
:01000300FEFE
:010005007B7F
:01000600BB3E
:01000800FCFB
:01000900BF37
:01000A00FFF6
:01000B00FFF5
:01000C00FFF4
:01000D00FFF3
:0200000400F00A
:0600000000F40100A00F56
:00000001FF
